:020000040000FA
:020000000528D1
:0800080015288312073099004E
:10001000850183169F011030850004309500403023
:1000200081008312FF30850051207D3033204E2027
:10003000003085007B303C205B3033205F30272050
:1000400085191228FF30850090308B002628F13E5C
:10005000A00020182B28A0182D28A0182F28FC3E1F
:1000600003182F280800FF3EA1005E3027206030D3
:100070002720A10B37280800FF3EA2006330332061
:100080005D302720633033205F302720A20B4228C9
:1000900008004D204E204E204D204E2051200000C3
:0400A0000000080054
:02400E00D33F9E
:00000001FF
